:100000000C94E7040C9404050C9404050C9404056A
:100010000C9404050C9404050C9404050C9404053C
:100020000C9404050C9404050C9437090C940405F5
:100030000C9404050C9404050C9404050C9404051C
:100040000C9404050C942B060C9404050C940405E4
:100050000C9404050C9404050C9404050C940405FC
:100060000C9404050C9404050C9404050C940405EC
:100070000C9404050C9404050C9404050C940405DC
:100080000C9404050C9404050C940405922077222A
:1000900097206222AE20AE20E820FD202F217E2175
:1000A000FA20772277221322252243225122772217
:1000B0007722772277227722772277227722772278
:1000C000772277227722662268226D224561737932
:1000D000436F6E74726F6C00204C430020504300DD
:1000E000696E636F6D70617469626C65204857005A
:1000F000312E342E340001020317180405061511A1
:1001000007080916120A000B0C13100F0E0D140E1F
:10011000111116111116100A00111111110E0011F2
:100120000E111111110E0011040A11111F110001FD
:100130000101050D1F0C04040E1F04041F0E040012
:10014000060917170906000006091214120906030A
:10015000070F1E1C181000030509121418100007C1
:100160000707070707070707050505050505071C16
:10017000101817150705071C101817110202021C8A
:10018000101812140605021C101817140601061C7C
:10019000101815150701011C101816110201061C74
:1001A000101816110204071C101812160202070478
:1001B0000A110A0A0E00000C17141714170C001C61
:1001C000101810160505051F0A0A0A0A0A1F000E54
:1001D00011111F1B1B1F0002060F1F0F0602000834
:1001E0000C1E1F1E0C08000E0E0E0E1F0E04000427
:1001F0000E1F0E0E0E0E00202020202020000020BA
:100200004D4D4920200000204D4D012020000020B0
:10021000444343202000002053544F5020000053FB
:10022000484F52542100002048414C542000000007
:10023000000000000000002050524F4720000052F4
:1002400045534554200000202054504D2000007E8E
:100250000E0E0E0E1B1B1C0E1B1B7E0E0E0E0E23F7
:100260002D004144523A20256C642020202020207B
:1002700020202020002D2D2D2D202000252D35641F
:10028000002533640020200102202020202020208F
:1002900000252D356400252D31312E31317300417B
:1002A00042434445464748494A4B4C4D4E4F5051B6
:1002B00052535455565758595A30313233343536D3
:1002C0003738392E2C3A2D2B232F3D3C7C3E2000F5
:1002D0004D4D20492020313420004D4D2049202013
:1002E000323761004D4D20492020323762004D4D9C
:1002F00020012020313420004D4D200120203237B4
:1003000061004D4D200120203237620044434320DC
:100310002020313420004443432020203238200064
:10032000444343202031323820004C6F636D656EAA
:100330007500000000000000000044434320686F87
:100340006F666473706F6F7200004C434420766573
:10035000726C69636874696E67004C6F6B436F6E93
:1003600074726F6C00000000000045786974000032
:10037000000000000000000000004B69657A656E17
:100380002000000000000000000044617461666FFE
:10039000726D61740000000000004E61616D2020EC
:1003A00020202020000000000000496E766F65725A
:1003B0002020202000000000000031323846532069
:1003C0004D6F64650000000000004D656E75204CA7
:1003D0006F636F0000000000000050726F67726171
:1003E0006D6D6174696F6E0000004C756D696E6FA4
:1003F000736974650000000000004C6F6B436F6E02
:1004000074726F6C00000000000045786974000091
:100410000000000000000000000053656C6563747C
:10042000696F6E20000000000000466F726D6174FD
:1004300020646F6E6E65657300004E6F6D20202026
:1004400020202020000000000000536169736965CE
:1004500020202020000000000000313238465320C8
:100460004D6F64650000000000004C6F6B204D650F
:100470006EFC00000000000000004443432048617F
:10048000757074676C65697300004C434420426565
:100490006C6575636874756E67004C6F6B436F6E47
:1004A00074726F6C000000000000457869740000F1
:1004B0000000000000000000000041757377E46850
:1004C0006C656E20000000000000446174656E667B
:1004D0006F726D617400000000004E616D65202038
:1004E0002020202000000000000045696E74726129
:1004F00067202020000000000000313238465320E1
:100500004D6F64650000000000004C6F636F6D6FFD
:1005100074697665206D656E7500444343204D61B6
:10052000696E20547261636B00004C434420626129
:10053000636B6C696768740000004C6F6B436F6E8F
:1005400074726F6C00000000000045786974000050
:100550000000000000000000000053656C6563743B
:10056000200000000000000000004461746120666B
:100570006F726D617400000000004E616D65202097
:1005800020202020000000000000456E74727920B9
:100590002020202000000000000031323846532087
:1005A0004D6F6465000000000000202D2D2D2D00F2
:1005B00025357500536F6674772E205600312E3422
:1005C0002E34005365724E722E2025386C75003A19
:1005D000200025357500253364002534643A200059
:1005E0002D2D2D0025336400204F4B20202020008E
:1005F0002020202020202000696E636F6D706174C0
:100600002E20466F726D617400496E636F6D702E9F
:1006100020466F726D6174202000466F726D6174A8
:1006200020696E636F6D7061742E00696E6B6F6D03
:100630007061742E20466F726D6174002E2E2E2014
:1006400077616974696E67202E2E2E2000233D6429
:10065000656C657465000000000000000000286EF5
:100660006F20656E74727929000000000000002E72
:100670002E2E2064656C6574696E67202E2E2E0008
:10068000206661756C74000000000000000000002E
:100690000020444343206F6E6C792100000000006D
:1006A000000020707265737320474F206669727373
:1006B0007400002A3D43616E63656C2020200000B9
:1006C000000000002070726F6772616D696E6700D4
:1006D00000000000002D73686F72742063697263FC
:1006E0007569742D2000206E61746976652028314B
:1006F0003A312920202000206C696E656172202823
:10070000323A3129202020002070726F67726573A1
:100710007369766520202020002E2E2E20776163BD
:100720006874656E202E2E2E2000233D776973732A
:10073000656E000000000000000000286765656E1F
:1007400020696E766F65722900000000202E2E2E23
:100750002077697373656E202E2E2E000020666F41
:10076000757400000000000000000000000020413F
:100770006C6C65656E20444343210000000000203E
:10078000707265737320474F20666972737400003E
:100790002A3D2041666272656B656E0000000000B4
:1007A000002050726F6772616D6D6572656E00003A
:1007B00000002D2D4B6F7274736C756974696E67D0
:1007C0002D2D00206E61746976652028313A31291B
:1007D00020202000206C696E6561722028323A3139
:1007E00029202020002070726F677265737369760C
:1007F00065202020200050617469656E74657A0060
:1008000000000000000000233D7375707072696D78
:100810006572000000000000766964650000000059
:1008200000000000000000000053757070726573D6
:1008300073696F6E000000000000204572726575DC
:10084000720000000000000000000020444343202C
:10085000756E697175656D656E74000020707265E6
:10086000737320474F20666972737400002A3D41FC
:1008700062616E646F6E2020000000000000205056
:10088000726F6772616D6D6174696F6E0000002D2B
:10089000436F7572742D636972637569742D2000DE
:1008A000206E61746976652028313A312920202034
:1008B00000206C696E6561722028323A312920204F
:1008C00020002070726F67726573736976652020EF
:1008D0002020002E2E2E2077617274656E202E2E21
:1008E0002E202000233D4CF6736368656E000000E7
:1008F0000000000000286B65696E2045696E747207
:10090000616729000000202E2E2E206CF67363688C
:1009100065202E2E2E2000204665686C6572000032
:100920000000000000000000206E75722066FC725E
:100930002044434321000000002065727374204767
:100940004F206472FC636B656E002A203D2041627B
:1009500062727563680000000000002050726F67CB
:1009600072616D6D696572756E6700002D2D204B8B
:1009700075727A7363686C75DF202D2D00204E61CF
:100980007469762028313A31292020202000204C1B
:10099000696E6561722028323A31292020200020BA
:1009A00050726F6772657373697620202020200073
:1009B0005B6E6F206D6573736167655D005B756E5F
:1009C0006B6E6F776E206572726F725D000011241E
:1009D0001FBECFEFD0E1DEBFCDBF11E0A0E0B1E0A0
:1009E000ECEAF0E500E00BBF02C007900D92A633E1
:1009F000B107D9F713E0A6E3B1E001C01D92AC3511
:100A0000B107E1F70C943E050C94000081E080935F
:100A100037010895482F90913601981731F096309C
:100A200021F0953029F4863019F080E090E00895A7
:100A300040933601453021F460E280E00E94BA2202
:100A400040913601463021F460E280E00E94BA22F3
:100A50000E94060581E090E0089508958091360196
:100A6000992708950E945C200E94171280913701F7
:100A7000882311F40E946D0CA8950895CFEFD0E162
:100A8000DEBFCDBF0E94D51D0E94E6050E940C0668
:100A900078940E94B5080E94FB1DFC0184810E948D
:100AA000D50C6CEC70E082E00E94330D0E94111EA8
:100AB000823021F00E94111E813019F468ED70E03F
:100AC00012C00E94111E803819F46CED70E00BC04A
:100AD00060E081E00E94830B60EE70E082E00E94A3
:100AE000330DA895FECF82E00E94330D60E081E0D7
:100AF0000E94830B66E582E00E94DA0C60EF70E0F2
:100B000082E00E94330D0E94FB1D8C0181E00E9457
:100B10007A0A882319F081E00E94FE1D82E00E947B
:100B20007A0A882319F080E00E94FE1D83E00E946B
:100B30007A0A882319F082E00E94FE1D84E00E9458
:100B40007A0A882329F083E00E94FE1D01C0A8953F
:100B50000E947B1F8823D9F3F80181859285892B18
:100B6000C9F00E94C70DEC014A969E012B5E3F4FD3
:100B7000AC01B901F801818592850E94C023BC01B6
:100B8000892B29F0F80181859285888F998F6115CD
:100B9000710519F4F801628173818FEF0E94761E4E
:100BA00081E011C00E944D120E942F0BFFEF8F3F7A
:100BB0009F07C1F70E943205809137018823A1F376
:100BC0001092370180E00E94560FEECF8FE78ABB6C
:100BD0001BBA80E187BB18BA80EF84BB8FEF85BB5F
:100BE0008BEB81BB8CEC82BB82E082B987EF83B94F
:100BF00087E78093610081EF809362008FE18093AB
:100C0000640089E1809365000E94EF09A89588E15E
:100C100081BD8CE081BD08950E94031E9B01AC0143
:100C200093E0E92FFF27EE5BFE4F822F8F778083C3
:100C300087E056954795379527958A95D1F7915036
:100C400097FFEFCF87B3807F87BB88B3807F88BB58
:100C500084EE8DB908951F920F920FB60F92112452
:100C60002F933F934F935F936F937F938F939F93B4
:100C7000EF93FF9380910001909101018F5F9F4F4F
:100C800071F0BB9A809100018FB9769B0BC0BB9825
:100C90001092380110923F0110923E0103C0BB98A0
:100CA0008FEF8FB97FB177FF7FC080914001909126
:100CB0004101892BE1F080913C018F5F80933C01E1
:100CC00080913C01803210F010923C0190913C01E7
:100CD00080913D01981759F480913D018F5F809379
:100CE0003D0180913D01803210F010923D018091D4
:100CF0003E0190913F01815F924061F058F08091F8
:100D00003B018F5F80933B0180913B01843010F069
:100D100010923B01109241011092400110923F014C
:100D200010923E0160913401761721F481E08093A6
:100D3000380171C010923801472F55279A012F773B
:100D40003070862F99272817390721F07F3F11F03F
:100D50006F3F61F490913C0189E0989FC00111249C
:100D60008F529E4F90934101809340014F77507076
:100D7000862F99274817590709F04DC090913A01DD
:100D800080913B01981749F090913B0189E0989F31
:100D9000C00111248F509D4F02C088EC91E09093C8
:100DA0003F0180933E0137C020913801822F99275F
:100DB0008130910531F0813091056CF106975CF539
:100DC00016C02F5F20933801703419F41092390146
:100DD00022C0713411F481E007C0723411F482E052
:100DE00003C0733491F483E08093390114C0E22F7F
:100DF000FF2780913901992702968E179F0744F0AB
:100E0000E05CFE4F8081781719F01092380103C022
:100E10002F5F2093380180913801882339F4809125
:100E20003E0190913F01892B79F003C0872F9927CC
:100E30000DC0E0913E01F0913F0181919927F0931F
:100E40003F01E0933E0102C08FEF9FEF90930101BD
:100E5000809300018091400190914101815F924017
:100E600020F01092410110924001E0914001F09178
:100E70004101309729F07193F0934101E0934001D3
:100E8000FF91EF919F918F917F916F915F914F9122
:100E90003F912F910F900FBE0F901F901895DC017E
:100EA00080913A01282F332780913B0199270197A0
:100EB0002817390741F080913A01833039F4809145
:100EC0003B01882319F480E090E0089590913A0165
:100ED00089E0989FF0011124EF50FD4F98E08D912B
:100EE0008193915097FFFBCF80913A018F5F809360
:100EF0003A0180913A01843010F010923A0181E079
:100F000090E008950895FC01A8ECB1E098E081918B
:100F10008D93915097FFFBCF08959C0190913C01D8
:100F200080913D01981719F480E090E00895D9016F
:100F30002115310511F4C9010895F89490913D01EE
:100F400089E0989FF0011124EF52FE4F98E08191C3
:100F50008D93915097FFFBCF80913D018F5F8093E0
:100F60003D0180913D01803210F010923D01789456
:100F7000C9010895089500000000000000000895D0
:100F8000882341F0809165008460809365000E9411
:100F9000BB070895809165008B7F8093650008955D
:100FA00008951F93182F8AB3807F8ABB80E00E9428
:100FB000C00780916500826080936500112321F055
:100FC00080916500816003C0809165008E7F809371
:100FD00065000000000081E00E94C00719B380E0B6
:100FE0000E94C0071295107F0E94BB0781E00E94FB
:100FF000C00789B38F70182B80E00E94C007812F33
:1010000099271F91089580E00E94D107982F809121
:101010004901882331F497FD04C0892F8F7780938D
:101020004A01892F992787FD90958827990F881F56
:10103000992708959B01AC018091170390911803A3
:10104000A0911903B0911A0382179307A407B5075B
:10105000A0F08091170390911803A0911903B0910B
:101060001A03821B930BA40BB50B80509041A04038
:10107000B040A0F080E090E0089580911703909137
:101080001803A0911903B0911A03281B390B4A0BBE
:101090005B0B2050304F4F4F5F4F18F081E090E0D6
:1010A000089580E090E008950895EF92FF920F93E5
:1010B0001F93AA27BB27E0901703F0901803009115
:1010C000190310911A03E80EF91E0A1F1B1F01C015
:1010D000A895C801B7010E941A088823C9F31F9177
:1010E0000F91FF90EF9008950F931F93CF93C82F08
:1010F000162F042F809165008D7F8093650080E01E
:101100000E94C0078AB38F608ABB8BB3807F9C2FFD
:1011100092959F70892B8BBB112321F080916500E4
:10112000816003C0809165008E7F8093650081E0BF
:101130000E94C00780E00E94C007002329F088E0D9
:1011400090E00E9455080DC08BB3807FCF708C2B30
:101150008BBB0E94BB0781E00E94C007802F0E94CA
:10116000C007CF911F910F9108950F931F93CF93B5
:1011700088E290E00E94550841E060E080E30E9430
:10118000740841E060E080E30E94740841E060E0A0
:1011900080E30E94740841E060E080E20E947408ED
:1011A00088E20E94790B80E40E94790B8AE00E9419
:1011B0004A0B89E20E94790B8CE10E94790B82E54F
:1011C0000E94790B89E60E94790B84E70E94790BD3
:1011D00080E40E94790B85E10E944A0B88E20E941C
:1011E000790B80E40E94790B0E94C70D8C0101C02D
:1011F000A89590911B0380911C039817C9F70E9432
:101200000308C82F8823A1F781E00E94D1078A3004
:1012100021F481E0F80187A302C0F801C7A388E0A8
:101220000E94790B81E00E94790B86E00E94790B85
:101230008CE00E94790B60E0862F0E94830B6FEE9A
:1012400071E080E00E94B20C67EC71E081E00E94E6
:10125000B20C6FEC71E082E00E94B20C67EB71E0BF
:1012600083E00E94B20CCF911F910F9108951F92BD
:101270000F920FB60F9211242F933F934F935F93CA
:101280006F937F938F939F93AF93BF93CF93EF937E
:10129000FF9380914801882309F08FC081E08093FB
:1012A00048017894809146018F5F80934601809138
:1012B00046018370992781309105F9F082309105BC
:1012C0001CF4892B21F077C0039759F174C08091E9
:1012D000170390911803A0911903B0911A03019676
:1012E000A11DB11D8093170390931803A0931903B8
:1012F000B0931A030E94150B5EC080911703909162
:101300001803A0911903B0911A0381709070A07016
:10131000B070892B19F00E948D0A4DC00E944E0AB0
:101320004AC060914701662319F00E94030841C03A
:1013300090911B0380911C03981789F0C0911C03A6
:10134000EC2FFF27E55EFC4F2281CF5FC03108F014
:10135000C62F203829F580911B038C1719F480E0E3
:1013600090E027C0EC2FFF27E55EFC4F22812F3F46
:1013700019F420914A01206827FF02C060934901B7
:10138000822F9927807C90708034910519F481E038
:1013900080934901CF5FC03108F0C62F462F02C0AD
:1013A000462F61E0822F0E947408C0931C0381E0E5
:1013B00090E08093470110924801FF91EF91CF9107
:1013C000BF91AF919F918F917F916F915F914F915D
:1013D0003F912F910F900FBE0F901F901895109274
:1013E0007D0080B7877F80BF17BE11BE89E683BFAF
:1013F00082E085BD87B7806487BF0895EF92FF9232
:101400000F931F93AA27BB27E0901703F0901803B0
:101410000091190310911A03E80EF91E0A1F1B1FF1
:1014200002C00E943205C801B7010E941A08882331
:10143000C1F31F910F91FF90EF900895282F220F75
:1014400061112160822F83708150823028F424FF43
:1014500002C02E6001C0217F822F992708959091AC
:101460004D01E92FFF27E35BFE4F8283892F8F5FBA
:1014700080934D01883010F010924D0190914E01F3
:1014800080914D01981741F4892F8F5F80934E0111
:10149000883010F010924E01089508950F931F9315
:1014A00011B1812F8074682F80914B010E941E0A18
:1014B000082F80934B011078612F80914C010E947E
:1014C0001E0A80934C01007C807C003829F488231C
:1014D00039F0803C61F408C0003449F4803C11F4D8
:1014E00089E103C0882319F48AE10E942F0A1F9121
:1014F0000F910895893118F080E090E0089520E080
:1015000030E0E82FFF27E95AFE4F8081882311F051
:1015100021E030E0C90108950895FF920F931F93D1
:10152000CF9380917501E82FFF27E059FE4F00818E
:1015300013B31F7081B1880F880F8071182B10832F
:10154000FF248091750125E0829FF0011124EF0DA9
:10155000F11DEA50FF4FC49110FD31C000FF14C0CF
:10156000C63129F485E10E947A0A882331F48C2F50
:101570000E942F0AC93108F043C0EC2FFF27E95A17
:10158000FE4F81E080833CC0C931D0F5EC2FFF27AE
:10159000DF01A95ABE4F9C919F5F9C93992311F440
:1015A0009F5F9C937597329758F580916C018937AE
:1015B00038F180916D01893718F1822F1FC0C93130
:1015C00028F4EC2FFF27E95AFE4F108200FD18C0C7
:1015D0008C2F80680E942F0A0E942E05853081F48E
:1015E000C53121F486E10E947A0A05C0C63141F472
:1015F00085E10E947A0A882319F486E00E940A0590
:1016000016950695F39484E08F1508F09ACF809193
:1016100075018F5F80937501853010F01092750110
:10162000CF911F910F91FF90089590917501943083
:1016300029F485B3806F85BB97980895979A85B3F1
:101640008F7020E130E002C0220F331F9A95E2F73D
:10165000922F9095907F892B85BB08950895809156
:101660004D0120914E01821719F48FEF9FEF0895DD
:10167000E22FFF27E35BFE4F8281482F5527822F01
:101680008F5F80934E01883010F010924E01CA0196
:1016900008950895CF93C82F07C080911C03882315
:1016A00091F40E945C20A89580911B03282F33277A
:1016B00080911C03992701972817390791F380918E
:1016C0001B038F3051F3F89480911B03E82FFF2701
:1016D000E55EFC4FC28380911B038F5F80931B03E9
:1016E00080911B03803110F010921B037894CF91EE
:1016F00008951F93182F80E80E944A0B812F0E94A3
:101700004A0B1F9108958295880F880F807C860F61
:1017100080680E94790B08950E94830B8EE00E94DE
:10172000790B08958CE00E94790B0895FF920F9336
:101730001F93CF93F82E60913E0380913D030E944A
:10174000830BC0E00DE213E080913F03C81778F4EB
:10175000FF2021F0F80161918F0101C060E282E079
:101760000E94DA0CCF5F80913F03C81788F3CF91B6
:101770001F910F91FF900895909348038093470322
:10178000892B89F17093460360934503CB01AA2707
:10179000BB272091170330911803409119035091F2
:1017A0001A03280F391F4A1F5B1F209341033093F0
:1017B00042034093430350934403809140038E7F40
:1017C00080934003211531054105510561F42F5FD8
:1017D0003F4F4F4F5F4F209341033093420340935D
:1017E00043035093440308950895AF92BF92CF925C
:1017F000DF92EF92FF920F931F93CF93DF93D82E38
:10180000C62EEA018DE2E82E83E0F82E10924803FE
:101810001092470381E08D1568F1EFE0E61750F173
:101820004115510539F1FA0101900020E9F731978E
:101830000E2F041B013108F000E16C2D8D2D0E944C
:10184000830B5701002361F0102F8881F5018193EC
:101850005F018991682F82E00E94DA0C1150A9F78C
:10186000F701D08AC18A028B64EF71E086E99BE0C0
:101870000E94BC0BDF91CF911F910F91FF90EF90D1
:10188000DF90CF90BF90AF900895CF93DF93CDB707
:10189000DEB7A0970FB6F894DEBF0FBECDBF282FDE
:1018A000DE01119690E0FA014F5F5F4F849188232B
:1018B00021F08D939F5F9F31B0F31C92AE014F5F7B
:1018C0005F4F822F0E94F50BA0960FB6F894DEBFF3
:1018D0000FBECDBFDF91CF910895809147039091C6
:1018E0004803892BA9F160914103709142038091D3
:1018F0004303909144030E941A08882349F1809180
:101900004003E0914703F09148038170099580916D
:10191000400391E089278093400380914503909193
:1019200046039C0144275527809117039091180383
:10193000A0911903B0911A03820F931FA41FB51F22
:101940008093410390934203A0934303B0934403D5
:1019500008950895109248031092470381E00E9471
:10196000790B08950F931F93CF93DF93EB0188308A
:10197000B8F4992723E0880F991F2A95E1F780642E
:101980000E94790B07E010E0FE01219684910E94ED
:101990004A0B0150104017FFF7CF8FEF0E94790BD1
:1019A000DF91CF911F910F910895813308F080E36B
:1019B00081BF0895CF93C62F823009F052C067FFD0
:1019C0004DC00E94C70DFC0187A18823C1F0C43E11
:1019D00011F4C4E843C0C63F11F4C4E93FC0CC3F92
:1019E00011F4C1E83BC0C43C11F4CEE837C0C63D99
:1019F00011F4C9E933C0CC3D49F5CAE92FC0C43E52
:101A000011F4C1EE2BC0C63F11F4CFEE27C0CC3F7E
:101A100011F4C5EF23C0C43C39F467E271E084E0FF
:101A20000E94B20CC4E01AC0C63D39F46FE171E007
:101A300085E00E94B20CC5E011C0CC3D39F467E1ED
:101A400071E086E00E94B20CC6E008C0CF3D31F4E0
:101A50006FE071E087E00E94B20CC7E08C2F0E941B
:101A60004A0BCF9108951F93CF93DF93182FEB016B
:101A7000FB016491662349F0812F0E94DA0C2196C4
:101A8000FE018491682F8823B9F7DF91CF911F91D0
:101A900008951F93CF93DF93182FEB01888188233C
:101AA00041F08991682F812F0E94DA0C8881882368
:101AB000C1F7DF91CF911F9108951F93CF93DF93CB
:101AC000CDB7DEB7C055D0400FB6F894DEBF0FBE1D
:101AD000CDBF67961FAD679769968EAD9FAD69972D
:101AE000AE01475A5F4FBC01CE0101960E94E3242C
:101AF000BE016F5F7F4F812F0E94490DC05BDF4F9A
:101B00000FB6F894DEBF0FBECDBFDF91CF911F910E
:101B100008951F93CF93DF93CDB7DEB7C055D04064
:101B20000FB6F894DEBF0FBECDBF67961FAD6797A7
:101B300069968EAD9FAD6997AE01475A5F4FBC0164
:101B4000CE0101960E940C25BE016F5F7F4F812F51
:101B50000E94490DC05BDF4F0FB6F894DEBF0FBE89
:101B6000CDBFDF91CF911F910895823019F40E946B
:101B70002F0B08958FEF9FEF08950895E82FFF270B
:101B8000EF70F070E15BFD4F84919927089586E72F
:101B900091E0089580918A0182FF05C080917801CB
:101BA000909179010895809176019091770108953F
:101BB000089580918A01826080938A0108950F932D
:101BC0001F93CF93DF93C6E7D1E080918A019927D5
:101BD0008C010170107080FF03C080E090E021C094
:101BE00060917E0170917F018091800190918101CF
:101BF000611571058105910531F00E941A0888234D
:101C000011F4C8010EC01A821B82188E198E109210
:101C10007701109276011C8A1A8E0E94060581E0D7
:101C200090E0DF91CF911F910F9108959C018091D9
:101C3000780190917901892B11F4C90108952F70D1
:101C40003F7B77FD3064CB018F70907044E0880F4C
:101C5000991F4A95E1F7822B932B08950895FC0173
:101C600080917601909177012091780130917901EE
:101C7000E817F907F9F460938C01232BB1F08091F8
:101C80007C0190917D01F4E096958795FA95E1F7B6
:101C9000BC016F707070892F99278695869580FD9D
:101CA0007068CA010E94160E11C050937D014093C6
:101CB0007C0110C0E217F30779F460938C01BA013C
:101CC00080917C0190917D010E94160E90937D0180
:101CD00080937C010E940605089508959C01892B3C
:101CE00069F410928A0110927E0110927F01109285
:101CF0008001109281010E94DF0D089560938C0194
:101D000050937D0140937C018091170390911803BB
:101D1000A0911903B0911A0388519C4FAF4FBF4F48
:101D2000816080937E0190937F01A0938001B093A6
:101D3000810180918A0182FF09C081608B7F80933D
:101D40008A01309379012093780107C08E7F8093B8
:101D50008A0130937701209376010E940605089549
:101D6000089520918A012B7F216020938A0190930E
:101D700079018093780180917C0190917D010E948E
:101D8000160E90937D0180937C010E9406050895B4
:101D9000CF93DF93EB0180938B010E94BE0D809364
:101DA0008D01209759F040E951E060E070E0CE01EC
:101DB0000E94C023D0938F01C0938E010E9406051C
:101DC000DF91CF910895CF93C82F882319F067E84A
:101DD00071E002C067EA71E084E00E94B20CCC239B
:101DE00019F06FE771E002C06FE971E085E00E94D1
:101DF000B20CCC2319F067E771E002C067E971E02B
:101E000086E00E94B20CCC2319F06FE671E002C0AC
:101E10006FE871E087E00E94B20CCF910895CF93F4
:101E2000DF93C82FDD27C4FF02C083E001C085EA2D
:101E30000E944A0BC0FF02C084E001C085EA0E94F4
:101E40004A0BC1FF02C085E001C085EA0E944A0B2F
:101E5000C2FF02C086E001C085EA0E944A0BC3FFB0
:101E600002C087E001C085EA0E944A0BDF91CF9152
:101E7000089580939C010E9406050895882319F017
:101E80006FE471E002C067E571E082E00E94B20C8D
:101E900008950895882319F06FE571E002C067E6A0
:101EA00071E081E00E94B20C089508950F931F9392
:101EB000CF9306E711E0C0919C01CC2399F060E03C
:101EC00081E00E94830B8C2F81500E947D1DBC01FC
:101ED00082E00E94330D10929C0188EE93E00E94F4
:101EE000FE0902C0882319F00E94AA0C03C0682FC3
:101EF0000E94830B8091760190917701892BF9F0F4
:101F00000E94FB1DFC0182819381409176015091DA
:101F100077018417950749F42185328580918E01D8
:101F200090918F012817390751F042835383809194
:101F30008E0190918F01818792870E94A01D209130
:101F40007601309177012115310529F4F8012683B6
:101F50003783168A158A80918A0182FD0DC080918F
:101F6000860190918701A0918801B0918901009725
:101F7000A105B10519F105C06FE572E082E00E948C
:101F8000330D8091860190918701A0918801B091D5
:101F90008901BF93AF939F938F9382E692E09F93C3
:101FA0008F9382E08F930E94890D8DB79EB707961D
:101FB0000FB6F8949EBF0FBE8DBF42C021153105EC
:101FC00031F465E772E082E00E94330D18C03F9360
:101FD0002F938CE792E09F938F93C2E0CF930E9460
:101FE000890D80918A010F900F900F900F900F90A4
:101FF00080FF02C08C2F01C080E20E944A0BC0917A
:102000008B010E942E05863008F08150833061F4E8
:102010008C2F99278370907023E0880F991F2A9541
:10202000E1F789509E4F08C0992703E0880F991F58
:102030000A95E1F7895E9D4FBC0182E00E94330D55
:102040006CE080E00E94830B80918C0199278F7750
:1020500090709F938F9381E892E09F938F9382E09B
:102060008F930E94890D80918B01992783709070C6
:102070000F900F900F900F900F90019779F487E1D8
:102080000E947A0A882331F080E00E944A0B67E3BD
:1020900071E010C080E20E944A0B0FC080E00E94F5
:1020A0004A0B80918C0187FF03C06FEE71E002C084
:1020B00067EE71E080E00E94B20C0E942E05C82FEE
:1020C000813049F489E00E94481DAC0160E08C2F0A
:1020D0000E94450CEBC040E050E060E0862F0E947B
:1020E000F50BC0E080918A0187FF0EC080917801D6
:1020F00090917901892B39F480918B019927837014
:102100009070039709F4C1E060E081E00E94830BC6
:102110008091860190918701A0918801B0918901F9
:102120000097A105B10509F442C08DE00E947A0A2A
:10213000882329F48EE00E947A0A882381F185E8B9
:1021400092E09F938F93C2E0CF930E94890D8DE020
:102150000E947A0A0F900F900F90882379F06FE514
:1021600071E081E00E94B20C67E571E08C2F0E9463
:10217000B20C6CE271E08AE49FE00EC067E671E0A9
:1021800081E00E94B20C6FE471E08C2F0E94B20CCF
:102190006CE271E08EE39FE00E94BC0B87C087E099
:1021A0000E94481DBC0182E00E94330D44C0809112
:1021B000780190917901009769F19F938F9381E95C
:1021C00092E09F938F9382E08F930E94890D80917C
:1021D0007C0190917D0114E0969587951A95E1F721
:1021E000282F2F70892F9927869586950F900F900D
:1021F0000F900F900F9080FD2061822F0E940F0F93
:10220000CC2321F08CE30E944A0B15C080E20E948F
:102210004A0B13C080E991E09F938F9386E992E087
:102220009F938F9382E08F930E94890D0F900F9060
:102230000F900F900F90CC2361F4809182019091C8
:102240008301A0918401B09185010097A105B1059A
:10225000C9F08091780190917901892B99F480914E
:102260007C0190917D01A4E096958795AA95E1F770
:102270008F7080610E940F0F81E00E94E30E6FEA71
:1022800071E011C020917C012F7080917C019091B0
:102290007D0197FD2061822F0E940F0F80E00E9438
:1022A000E30E67EB71E083E00E94B20CCF911F91C7
:1022B0000F910895EF92FF920F931F93CF93DF93A7
:1022C000CDB7DEB726970FB6F894DEBF0FBECDBFF1
:1022D0008C0186E0FE01319611928A95E9F7F801AA
:1022E00020893189428953896281738121153105A1
:1022F0004105510509F483C06115710569F1E0805C
:10230000F180C701AA27BB2782179307A407B50747
:1023100041F0CB01AA27BB2782179307A407B50773
:10232000D9F4F80184898E7F848B80818F778983AB
:10233000EE0CEF2CEE1CFF08F1948E2D8F778A8324
:10234000AE014F5F5F4F65E080E00E944620F801DC
:102350001282138210821182D8018D919C919C016E
:1023600044275527F80180899189A289B389648916
:10237000281739074A075B0729F481E068276B7F34
:10238000648B44C06C7FF801648B108E118E128EAA
:10239000628D81E00E94830B80E00E94481DBC0199
:1023A00082E00E94330DF8018489992796958795DC
:1023B000969587959C012170307080FD14C08081B6
:1023C0009181009711F084839583F80122833383F0
:1023D0002683378320833183158A608971898FEF43
:1023E0000E94761E08C0F801408951896081718180
:1023F0008FEF0E94A51EF80184898B7F05C0672B93
:1024000021F4F80184898460848BF801108A118A90
:10241000128A138A26960FB6F894DEBF0FBECDBF80
:10242000DF91CF911F910F91FF90EF9008956091F0
:102430007E0170917F0180918001909181016115F1
:1024400071058105910561F00E941A08882341F009
:1024500010927E0110927F011092800110928101F2
:102460006091820170918301809184019091850136
:10247000611571058105910571F00E941A08882384
:1024800051F01092820110928301109284011092F7
:1024900085010E94060508950895CF92DF92EF927C
:1024A000FF920F931F93CF93DF93CDB7DEB72C9797
:1024B0000FB6F894DEBF0FBECDBFBC0186E7C82EB5
:1024C00081E0D82E86E0FE01319611928A95E9F7D7
:1024D00065317105DCF46F3071050CF05EC16A3056
:1024E000710509F4FEC16B3071053CF4611571058D
:1024F00009F492C177FD05C2BBC16C30710509F4C6
:10250000D4C06D3071050CF0EEC0E2C16B317105C5
:1025100084F469317105F4F46631710509F46CC114
:10252000663171050CF46AC16731710509F4AAC0FE
:10253000E8C16F3871054CF46D3871050CF0D3C0EB
:102540006A38710509F4C9C1DCC16739710509F43C
:10255000D6C1D7C1EE246931710511F401E0E02E36
:1025600010918C0100918D010E94FB1DFC01F780F0
:10257000EE20B1F00E942E05412F5527833041F403
:102580009A012F773070802F99272817390714F078
:102590009A0175C00E3711F4FF2071F41F5F26C039
:1025A000212F3327C9018F779070892B09F467C0D9
:1025B0000E37D9F4FF20C9F0212FEE2059F0F2E0B8
:1025C000FF1641F4812F99278F779070449714F468
:1025D0002F5F54C0EE2069F482E0F81651F4812F89
:1025E00099278F779070459754F41150212F3327F6
:1025F00046C0E1E0FE1619F4212F2E7F14C0812F72
:1026000099278F779070459714F0212F2E7F422FB6
:102610005527CA018F779070CF972CF04E535040BA
:102620004C7F242F225C211769F0EE2039F1F2E073
:10263000FF1609F5822F99278F779070CE97DCF0DF
:102640002F0F19C0EE2051F082E0F81639F4822FD6
:1026500099278F779070CE970CF02E5FEE2059F46B
:10266000E2E0FE1651F4822F99278F779070CF9772
:1026700024F0225002C02E5F01C022503327F60101
:10268000268B3DC180918B019927837090700197B3
:1026900029F467E371E080E00E94B20C80918C0124
:1026A0008095807880938C012AC180918A0187FF70
:1026B00013C08091780190917901892B69F0809104
:1026C0007C0190917D0120E030E482279327909354
:1026D0007D0180937C0113C180917C0190917D01EB
:1026E00020E030E883C086E017E0E12EF12CEC0E0C
:1026F000FD1EF70111928A95E9F78091860190916C
:102700008701A0918801B09189010097A105B105C9
:1027100009F441C0009186011091870101501040D9
:10272000000F111FCB018F7790700E9709F4016095
:1027300067FF16C01A8660E070E0CB010E94BC0BF8
:1027400067EC71E081E00E94B20C6FEC71E082E016
:102750000E94B20CF601108A118A128A138A02C0F2
:1027600081E08A87802F8F778F83000F012F001FD2
:10277000110B1195802F8F778887000F012F001F75
:10278000110B1195802F83708987A70166E080E087
:102790000E944620B4C067FDB2C0613171058CF063
:1027A0008091170390911803A0911903B0911A0317
:1027B0008C509E4FAF4FBF4FF60184879587A687F9
:1027C000B787962F9D5080918A0187FF04C06131A1
:1027D00071050CF49C5F21E030E002C0220F331F32
:1027E0009A95E2F780917C0190917D018227932751
:1027F000F6018683978383C043E005C080918A01F8
:1028000087FF04C042E060E280E003C040E060E295
:10281000842F0E94BA2273C080918A0187FF15C05D
:1028200080917A0190917B01009709F46AC0AA27F0
:10283000BB278093860190938701A0938801B09372
:102840008901C6010E945A115CC080918601909155
:102850008701A0918801B09189010097A105B10578
:1028600039F48FEF0E94121D81E00E94560F49C07B
:102870008091860190918701A0918801B091890192
:102880009C01AD01E3E0220F331F441F551FEA9561
:10289000D1F7280F391F4A1F5B1F280F391F4A1F06
:1028A0005B1FCB01AA2797FDA095BA2F280F391FD0
:1028B0004A1F5B1F2030F8E23F07F0E04F07F0E0CF
:1028C0005F07FCF4F601208B318B428B538B17C0D2
:1028D00086E791E00E945A1112C080918A018F7799
:1028E0000CC01092860110928701109288011092FC
:1028F000890180918A018B7F806880938A010E9480
:1029000006052C960FB6F894DEBF0FBECDBFDF9143
:10291000CF911F910F91FF90EF90DF90CF9008958E
:10292000FB0121E057FF04C020E0509541955F4F27
:102930008330910549F18430910534F4813091055B
:1029400091F0029729F12AC08430910519F005977A
:1029500061F024C081818F5F818399278417950757
:10296000ECF0222359F0118219C0818181508183BA
:1029700099278417950794F0222321F0842F815002
:1029800081830CC021830AC012821382168A06C07A
:1029900090E08281882309F491E0928380E090E0C6
:1029A00008950F931F93CF93DF938C010E94CA0D5C
:1029B000EC01009731F46AEA75E082E00E94330D81
:1029C0000FC09F938F9380EB95E09F938F9382E04E
:1029D0008F930E94890D0F900F900F900F900F9082
:1029E0000115110521F0B80182E00E94330DCE01DE
:1029F000DF91CF911F910F9108950F931F93CF9364
:102A0000DF93EC018B01009731F097FD35C0029701
:102A1000029790F52BC060E081E00E94830BF801E3
:102A20008281882359F464EB75E082E00E94330DC3
:102A30006DEB75E082E00E94330D18C00E94031E0A
:102A4000DC01CB01BF93AF939F938F9383EC95E011
:102A50009F938F9382E08F930E94890D8DB79EB7CD
:102A600007960FB6F8949EBF0FBE8DBF40E050E0B2
:102A7000B801CE010E94901480E090E0DF91CF91E8
:102A80001F910F9108958230910541F08330910597
:102A900041F440E050E00E94901403C08FEF9FEF9C
:102AA000089580E090E0089508952F923F924F920C
:102AB0005F926F927F928F929F92AF92BF92CF92CE
:102AC000DF92FF920F931F93CF93DF93CDB7DEB7C3
:102AD00026970FB6F894DEBF0FBECDBF8C015B0109
:102AE0000E94C70D6C010230110509F457C0033074
:102AF00011053CF401151105E9F00130110531F023
:102B0000CAC0063011050CF0C6C02CC0FC01F58807
:102B10002F2D269526952370F3E0FF2211F451E026
:102B2000F52E83E0F89EC0011124280F2350F501F3
:102B30002183B1C060E081E00E94830B8FEC95E0BF
:102B40000E94D114892B09F4A6C0F50191818AE075
:102B5000989FC001112480539D4FBC0182E00E94C8
:102B6000330D99C049E050E0B501C8010E949014AE
:102B7000F601808191818F3F910509F008F48BC0A7
:102B8000F5018181882311F486E08183F50181813B
:102B9000863008F080C088E081837DC0FC014280DF
:102BA00053804114510409F076C0F50182818823D5
:102BB00009F469C0F601808091808114910409F4C0
:102BC0006AC0F5012181822F63E00E942828F82E37
:102BD000F394822F0E942828892F9927880F991F04
:102BE000880F991FF82AF601208C318C3AE1632E68
:102BF000712C6C0C7D1C8501065F1F4FB301C80151
:102C00000E94DC2486E0FE01319611928A95E9F754
:102C1000882D8F778983C401880F892F881F990B8E
:102C200091958F778A83FFE7FF22FB82AE014F5F8A
:102C30005F4F64E08FEF0E94462060E081E00E94D9
:102C4000830B80E00E94481DBC0182E00E94330D8E
:102C5000A20160E0C2010E946E0EB4018FEF0E94DB
:102C6000761EB801C3010E94DC242114310459F0FE
:102C70009301F601458960817181C1010E9403239E
:102C8000F601808F918F90E0F5018281882309F40D
:102C900091E0F501928380E090E026960FB6F894DB
:102CA000DEBF0FBECDBFDF91CF911F910F91FF907F
:102CB000DF90CF90BF90AF909F908F907F906F905C
:102CC0005F904F903F902F900895482F30E0832FD2
:102CD000992787FD9095FC01E156FD4F249124171B
:102CE00029F03F5F222399F78FEF9FEF0895089512
:102CF000EF92FF920F931F93CF93DF93EB018230FC
:102D0000910509F486C08330910534F4009709F4E5
:102D10003EC0019769F0BAC08430910509F443C000
:102D2000843091050CF470C0059709F456C0AEC00C
:102D30000E94C70D8C01FC0180819181892B09F4CF
:102D4000A5C06AE1E62EF12CE00EF11E8E01065FB1
:102D50001F4F65960C171D07B8F4F7018081882373
:102D600039F00E94651687FD03C0F701808101C01C
:102D700080E2F80181938F01F7018081882351F36C
:102D80000894E11CF11CE6CFF80110827FC00E947C
:102D9000D11460E081E00E94830B2A96BE0182E09C
:102DA0000E94490D73C08981FB01E80FF11DEF01FD
:102DB0002A9682850E9465168F5FE82FFF27E7FD20
:102DC000F095E156FD4F8491882319F4EFE9F2E084
:102DD0008491992787FD909515C08981FB01E80FA3
:102DE000F11DEF012A9682850E946516181614F0CF
:102DF0008FE201C08150E82FFF27E7FDF095E156F3
:102E0000FD4F8491888342C049E050E00E949014B5
:102E10003DC00E94C70D8C01FC0182819381892BEA
:102E2000A9F59A81992349F489E08B8381E0888F01
:102E300099839F8B8A838E8B29C089818F5F898339
:102E40008F8B8B3018F11B821A821E8A8CE09801BE
:102E5000265E3F4FD901FE013A9601900D928A9568
:102E6000E1F7F801808D918D009731F045896081FF
:102E700071810E94032307C0A901F801658980813F
:102E800091810E94B823F801808F918F80E090E0BB
:102E9000DF91CF911F910F91FF90EF9008958F9246
:102EA0009F92BF92CF92DF92EF92FF920F931F9368
:102EB000CF93DF93CDB7DEB727970FB6F894DEBF79
:102EC0000FBECDBF9C018B018230910509F455C026
:102ED000833091052CF40097C1F0019759F0C8C0D8
:102EE00084309105D9F1843091050CF441C00597E7
:102EF000C9F1BEC04BE050E060E270E0C8010A9644
:102F00000E94D524F801158AB3C0FB018281882371
:102F100009F4AEC08181882309F4AAC0065F1F4F5F
:102F2000A801B90199270E94C0239F938F9382ED36
:102F300095E09F938F93F2E0FF2EFF920E94890D00
:102F400060E081E00E94830BB8018F2D0E94490D43
:102F50000F900F900F900F900F908AC0FB0181810E
:102F6000992721C0FB01818199270E94AD241DC0B2
:102F700049E050E00E9490147BC090E0FB01828108
:102F8000882309F491E0F80192830E94C70D7C0127
:102F9000F801B280BB2061F0FC01808D918D00971B
:102FA00011F0808D02C00E94A924F801818360C0C5
:102FB000EAE08E2E912C800E911EF8018181A401F1
:102FC000BE01695F7F4F99270E94C0236C01F70102
:102FD0001282138210821182BC018FEF0E94761E32
:102FE000F70180819181892B81F186E0FE01319684
:102FF00011928A95E9F78C2D8F778983C601880F06
:10300000892F881F990B91958F778A838F818F776E
:103010008B83AE014F5F5F4F64E08FEF0E944620CD
:103020006B2D81E00E94830B8B2D0E94481DBC01FB
:1030300082E00E94330D40E050E06B2DCA010E94F7
:103040006E0EB6018FEF0E94761EF701808191818E
:10305000892B59F0B401C7014A960E94DC24F8017B
:1030600081819927F701808F918F8FEF9FEF02C0A9
:1030700080E090E027960FB6F894DEBF0FBECDBF7C
:10308000DF91CF911F910F91FF90EF90DF90CF9044
:10309000BF909F908F9008950F931F93CF93DF93CE
:1030A000EC010E94C70D8C01209719F02297C9F0FE
:1030B0003DC0CE010E94D114892BC1F160E081E0B6
:1030C0000E94830BF801808D918D892B11F081E096
:1030D00001C082E00E94481DBC0182E00E94330DC5
:1030E00025C0FC01C281D381209701F580819181A7
:1030F000892BE1F0808D918D892BC1F060E081E01A
:103100000E94830B83E00E94481DBC0182E00E9464
:10311000330D84EF91E00E94FE09F801808D918DBE
:103120000E94D922F801C08FD18F128E80E090E0EA
:10313000DF91CF911F910F910895CF93DF93EB0112
:103140008230910561F1833091052CF4009781F074
:10315000019729F034C0863091058CF51BC00E9480
:10316000FB1DFC0187818983833048F1198227C0C8
:1031700060E081E00E94830B8981865F0E94481D88
:103180009F938F9382E08F930E94890D0F900F90F1
:103190000F9015C043E050E00E94901410C08A8147
:1031A000882339F00E94FB1D2981FC0127830E949E
:1031B000A01D90E08A81882309F491E09A8380E041
:1031C00090E0DF91CF9108951F93CF93DF93EB01B0
:1031D0008230910509F440C0833091052CF40097AA
:1031E00089F0019731F04CC0863091050CF048C051
:1031F0002EC00E94FB1DFC01848163E00E942828F0
:1032000089833EC060E081E00E94830B898113E0E6
:10321000819F802D11240E94D50C82E090E00E94B5
:10322000FE0981B7612F0E942828898399279F93DF
:103230008F9386ED95E09F938F9382E08F930E940A
:10324000890D0F900F900F900F900F9019C04FEEB7
:103250005FEF0E94901414C08A81882359F00E9465
:10326000FB1D398123E0329F90011124FC0124834E
:103270000E94A01D90E08A81882309F491E09A833E
:1032800080E090E0DF91CF911F910895CF92DF927F
:10329000EF92FF920F931F93CF93DF93CDB7DEB7DB
:1032A00026970FB6F894DEBF0FBECDBF8C017B0111
:1032B0000E94C70D6C01FC0180819181892B31F046
:1032C0008589992783709070039731F060E081E0E1
:1032D0000E94830B85E00DC00E942E05833081F093
:1032E0000E942E05823061F060E081E00E94830B35
:1032F00086E00E94481DBC0182E00E94330D02C19D
:103300000230110509F49DC0033011053CF401158C
:10331000110539F10130110571F0F4C004301105C7
:1033200009F48DC0043011050CF4E6C00530110518
:1033300009F4DEC0E7C08EEF9FEFF701818F928F17
:103340002091A5013091A601C901019780509440B8
:1033500020F4F70124833583D5C0F7010483158356
:10336000D1C060E081E00E94830BF7018281882355
:1033700011F488E0BECF60E081E00E94830BF7018A
:10338000848195819F938F938AED95E09F938F938E
:1033900012E01F930E94890D0F900F900F900F90D5
:1033A0000F90F7018381843059F480EE95E09F936C
:1033B0008F931F930E94890D0F900F900F9011C053
:1033C000F701808599279F938F9384EE95E09F93D3
:1033D0008F931F930E94890D0F900F900F900F9065
:1033E0000F90F701818D928D97FD03C068EE75E017
:1033F0000AC08E5F9F4F19F460EF75E004C084E04F
:103400000E94481DBC0182E00E94330D81E0F7015B
:10341000808F868B83819927813091056CF0833072
:10342000910524F00497029738F402C083E001C0AC
:1034300088E0F701878B66C0F701168A63C084E0D5
:1034400058C0F701828124813581882389F441E0C5
:10345000438380E094E086839783821793072CF45C
:1034600081E090E0F70184839583F70142834AC0AD
:103470003093A6012093A50121153105C9F1F7016B
:10348000838181508230A0F1F60180818F7789831A
:1034900080819181880F892F881F990B91958F7753
:1034A0008A83F701848181508F778B83215030404C
:1034B000220F232F221F330B322F37702085822FAC
:1034C00099278078907095958795382B3C832F7736
:1034D0002D831E82AE014F5F5F4F67E08FEF0E942A
:1034E0004620F70113820E94920B8FEF9FEF0CC0D2
:1034F00081E0F701838306C040E050E0B701C801D6
:103500000E94901480E090E026960FB6F894DEBFFB
:103510000FBECDBFDF91CF911F910F91FF90EF9024
:10352000DF90CF900895CF92DF92EF92FF920F93AA
:103530001F93CF93DF937C01C62F0E94AA0C0E9499
:10354000FB1D6C01CB3008F06FC085E0C89F800187
:1035500011240E5F1E4FF7018281882311F080E055
:1035600001C082E00E944A0BF601858199278130D3
:103570009105B1F0823091051CF4892B39F031C0EE
:1035800082309105B9F00397F9F02BC08C2F992761
:1035900054E0880F991F5A95E1F7865F9A4F1DC036
:1035A0008C2F992744E0880F991F4A95E1F7865997
:1035B0009B4F13C08C2F992734E0880F991F3A95A1
:1035C000E1F786539C4F09C08C2F992724E0880F80
:1035D000991F2A95E1F7865D9C4FBC0182E00E940D
:1035E000330DE8018C8187FD0BC060E081E00E9413
:1035F000830B8C810E94481DBC0182E00E94330D28
:10360000E801EA81FB81309721F0B70180E090E08A
:103610000995F7018689882329F06789808D0E94A2
:103620008C0B02C00E94920BDF91CF911F910F91E2
:10363000FF90EF90DF90CF90089560E0E2E0F1E03E
:10364000482F552747FD509520E030E0808199278D
:103650008417950711F4C90108956F5F2F5F3F4FDD
:1036600035966A3098F38FEF9FEF08950895BF92D3
:10367000CF92DF92EF92FF920F931F93CF93DF933E
:10368000CDB7DEB76B970FB6F894DEBF0FBECDBFD8
:10369000B82E29E0281718F480E090E0B3C16E013D
:1036A0000894C11CD11C8BE1F60111928A95E9F7AF
:1036B000A89585E0B89EF0011124EE5FFE4F0280D0
:1036C000F381E02D309721F0B60181E090E009957B
:1036D0006B2DC6010E94931A0E94320515E0B19E1F
:1036E0007001112482E091E0E80EF91E0E942F0B78
:1036F000AC018B30910509F497C08C30910534F4FE
:1037000097FDEACF0A970CF4FEC0D6C08731910529
:1037100009F48AC08831910524F4459709F46BC1F6
:10372000DBCF8931910519F04A9751F1D5CFF601D8
:103730008281882381F0F7012281338121153105AF
:1037400031F0BE016F5F7F4F84E090E051C1F60120
:1037500081818F5F28C0F601868BF7019081F8E0A8
:10376000FB1534F0F7018581891711F4B39431C04A
:10377000892F0E941D1B682F772767FD709540C019
:10378000F6018281882389F0F70122813381211596
:10379000310531F0BE016F5F7F4F85E090E028C1B9
:1037A000F60181818150818329C1F601868B6B2DC1
:1037B000F7019081BB2091F02BEF3FEFE20EF31E5B
:1037C000F701808125E030E0E20EF31E891731F425
:1037D000BA946B2D772767FD709512C038E03B15C2
:1037E00064F0D7011596F7018581891731F46F5F71
:1037F00069301CF415968C91F8CF772767FD70958A
:10380000B62E85E0689FF0011124EE5FFE4F028026
:10381000F381E02D309709F4F1C0BE016F5F7F4F57
:1038200081E090E00995EAC0F7019181992361F167
:10383000092F112702561E4FF801808118162CF00F
:10384000892F0E941D1BF8018083F7018181E82FD9
:10385000FF27E256FE4F80810E94371B282F332717
:1038600027FD3095F7018181E82FFF27E256FE4FB3
:10387000C90137FF04C088279927821B930B8083D7
:1038800037FFBCC0B1943AC0F701228133812115C2
:10389000310551F0BE016F5F7F4F82E090E0F9018A
:1038A000099599237CF319C0F6018281882309F4D4
:1038B00091E0F6019283A2C0F60182818823F1F0A3
:1038C000F7012281338121153105A9F0BE016F5F17
:1038D0007F4F83E090E0F9010995F601828188230A
:1038E00009F08CC0F70122813381BE016F5F7F4FE9
:1038F00081E090E07DC0F601128280C08B2D992777
:1039000087FD90957FC0F6018381992784309105CA
:1039100009F446C0853091054CF48230910539F1A7
:103920008330910584F4019771F068C08830910567
:1039300051F0893091051CF40597A9F15FC00997F2
:1039400009F444C05BC0F60186819781892B21F47C
:103950008FEF9FE786839783F6018681978184178F
:1039600095070CF44BC01482158282E08383F60124
:10397000848195819C0163E0220F331F6A95E1F7F2
:10398000280F391F280F391F240F351F37FD36C068
:1039900086819781821793078CF1248335832EC00B
:1039A000F60110861383F60190858AE0989F9001B6
:1039B0001124240F351F2F3F310509F008F420870B
:1039C0008EEF9FEFF601818F928F18C0F6018181F3
:1039D000E80FF11D842F805D8287F70122813381FA
:1039E0002115310559F0BE016F5F7F4F82E090E0F5
:1039F000F901099503C080E00E940A056B2DCE01F4
:103A0000019668CE6B960FB6F894DEBF0FBECDBFA1
:103A1000DF91CF911F910F91FF90EF90DF90CF90AA
:103A2000BF900895CF93C82F0E94111E803871F166
:103A30006FE271E080E00E94B20C67E371E082E027
:103A40000E94B20C80919E018A3010F010929E016B
:103A5000C7FD04C08C2F0E94371B0EC080919E01B1
:103A60000E94371B992787FD909597FF03C090957B
:103A700081959F4F80939E016FEE71E080E00E94E0
:103A8000B20C6FEC71E082E00E94B20CCF9108950D
:103A9000CF93C82F8D3018F080EB99E02CC00E9496
:103AA000FB1DFC01858199278230910581F08330CF
:103AB00091051CF4019721F018C0039779F015C007
:103AC00081E1C89FC00111248D52974F14C081E13C
:103AD000C89FC00111248A50984F0DC081E1C89F32
:103AE000C0011124875E984F06C081E1C89FC001C4
:103AF0001124845C994FCF910895882319F08DEBA0
:103B000099E008950E94FB1DFC0185819927823070
:103B1000910561F0833091051CF4019721F00CC0F0
:103B2000039739F009C08BE296E008958AE196E0A8
:103B3000089589E096E0089588EF95E00895089546
:103B4000EF92FF921F93CF93DF9387EAE82E81E0F5
:103B5000F82EC0E0D0E01FE1CE010E94B124F701B1
:103B600061917F01861719F0CE010E94CA24A895A1
:103B70001150219617FFF0CFDF91CF911F91FF9049
:103B8000EF9008959091AC01943008F091E08FE0AF
:103B9000E7EAF1E011928A95E9F788E18093AB01B9
:103BA0009093AC010E94A01D089540E250E060E0B7
:103BB00070E087EA91E00E94B9248091A901909178
:103BC000AA018F5F9F4F11F40E94C21D8091AC012A
:103BD000843010F01092AC018AEF9FEFA1E0B0E0CA
:103BE000ABBFFC0187918F3F21F0882311F08093B8
:103BF0006F000895089587EA91E008958093AC01DD
:103C00000E94A01D08958CEF9FEFA1E0B0E0ABBF34
:103C1000FC0187919791A791B691B070BC01CD013D
:103C200008958FEF9FEFA1E0B0E0ABBFFC0187915B
:103C3000823011F4079B80E899270895FC0184895C
:103C40009927969587959C012170307080FD02C060
:103C5000C901089580819181009711F081E090E081
:103C600008950895FC0182819381009711F081E00D
:103C700090E008950895CF92DF92EF92FF920F9314
:103C80001F93CF93DF93C82E7B01EA010E94C70DDB
:103C90008C01209711F1DD24A7016C2D80E00E949A
:103CA00046208AE08093490302C00E943205C80181
:103CB000FE010995882321F4809149038823A9F7FF
:103CC0000E946E1F8111DD24C801FE010995882321
:103CD00021F4D39487E08D15F8F6DF91CF911F91F1
:103CE0000F91FF90EF90DF90CF900895CF93DF93E7
:103CF000CDB7DEB726970FB6F894DEBF0FBECDBFA7
:103D000061157105C9F086E0FE01319611928A9520
:103D1000E9F7862F8F778983660F672F661F770BEA
:103D20007195862F8F778A834EE15EE1BE016F5FCA
:103D30007F4F81E00E943B1E26960FB6F894DEBFAF
:103D40000FBECDBFDF91CF910895CF93DF93CDB755
:103D5000DEB726970FB6F894DEBF0FBECDBF611554
:103D6000710539F14115510521F186E0FE013196C9
:103D700011928A95E9F7862F8F778983660F672FCF
:103D8000661F770B7195862F8F778A83842F8F77A5
:103D90008B83440F452F441F550B5195842F8F77EC
:103DA0008C8342E35EE1BE016F5F7F4F82E00E9441
:103DB0003B1E26960FB6F894DEBF0FBECDBFDF9137
:103DC000CF910895F894FFCFFC0180E0482F57E091
:103DD0002191282780E0922F96958F5F20FF03C0C6
:103DE000292F252701C0292F8830A8F33327822FB8
:103DF0004F5F483068F327FD8095992708950F930A
:103E00001F938C010E94E41EF8019085891719F018
:103E100080E090E002C081E090E01F910F91089552
:103E2000EF92FF920F931F93CF93DF93CDB7DEB73F
:103E300029970FB6F894DEBF0FBECDBF9C018091CD
:103E4000340180687E010894E11CF11C898383E0C1
:103E5000F701818387010E5F1F4F822F8F77F80153
:103E60008193220F232F221F330B3195822F8F77BF
:103E70008193862F8F7781938F01CA01892F99278C
:103E8000869586958F73808367FF02C080648083E8
:103E90000F5F1F4FCA0123E0969587952A95E1F79A
:103EA0008F77F8018193842F8295807F8F7781931C
:103EB0008F01C7010E94E41EF8018083C7010E94A0
:103EC000830729960FB6F894DEBF0FBECDBFDF91F2
:103ED000CF911F910F91FF90EF9008958091C701AE
:103EE000882319F480E090E008951092C70181E0E2
:103EF00090E008950895EF92FF920F931F93CF9350
:103F0000DF93CDB7DEB729970FB6F894DEBF0FBEAB
:103F1000CDBF0E94031E7B018C0165C0A8958A81DC
:103F2000843009F060C0CE0101960E94FF1E8823F4
:103F300009F459C0D801C7018F779070A070B07094
:103F40002E8133274427552782179307A407B507E7
:103F500009F049C0D801C70180789F73A070B07084
:103F600027E0B595A795979587952A95D1F72D8147
:103F700033274427552782179307A407B50799F5D8
:103F8000D801C7018070907CAF71B070FEE0B5952C
:103F9000A79597958795FA95D1F72C8133274427D4
:103FA000552782179307A407B507E9F4D801C7017D
:103FB00080709070A07EB070E5E1B595A79597955B
:103FC0008795EA95D1F72B81332744275527821708
:103FD0009307A407B50739F489818F77809334015B
:103FE00081E090E007C0CE0101960E948D07009706
:103FF00009F094CF29960FB6F894DEBF0FBECDBF5F
:10400000DF91CF911F910F91FF90EF9008958091D4
:104010003401992708950F931F93CF93DF93CDB762
:10402000DEB729970FB6F894DEBF0FBECDBFFA01F9
:10403000A89580913401806889836A838E010D5F21
:104040001F4F95E0309729F081918F77D8018C939D
:1040500002C0D8011C9291500F5F1F4F97FFF2CF03
:10406000CE0101960E94E41EF8018083CE010196E4
:104070000E944F07992729960FB6F894DEBF0FBE0E
:10408000CDBFDF91CF911F910F9108950F931F9393
:10409000CF93DF93082F162FEA0102C00E9432054A
:1040A000AE01612F802F0E940B208823B9F3DF918E
:1040B000CF911F910F9108959F92AF92BF92CF928F
:1040C000DF92EF92FF920F931F93CF93DF93CDB7C1
:1040D000DEB72F970FB6F894DEBF0FBECDBF31C24B
:1040E000CE0101960E94FF1E882309F42AC26E01A8
:1040F0000894C11CD11C0E94C70D5C01F6016181AE
:10410000862F9927AA27BB27FC013397E032F105B8
:1041100008F0EDC1EA5BFF4FEE0FFF1F0590F49131
:10412000E02D0994F60182810E940A05E0C1F601A2
:104130008281282F3327838199279695982F882766
:1041400097958795282B392BD5018D919C918217B6
:10415000930709F0CCC10E94DF0DC9C1F60182812D
:10416000A82FBB27838199279695982F8827979505
:104170008795A82BB92B8581282F3327A901542F88
:104180004427550F550F868199278F77907013E03C
:10419000880F991F1A95E1F7482B592B878199278A
:1041A0008077907074E0959587957A95E1F7482B24
:1041B000592B683029F4BA01CD010E94B10E97C184
:1041C000F601648126FD6068CD010E946E0E8FC1EC
:1041D000F6018581282F3327868199279695982F78
:1041E000882797958795282B392BB90184810E94C0
:1041F000C80E7DC10E94D90D7AC1F6018281A82F17
:10420000BB27838199279695982F8827979587951F
:10421000A82BB92B8581282F3327A901542F442798
:10422000550F550F868199278F77907003E0880F7F
:10423000991F0A95E1F7482B592B87819927807799
:10424000907014E0959587951A95E1F7482B592BB6
:10425000648126FD6068CD010E942F0E48C1F501E2
:10426000808D918D892B41F0A8E09A2E808D8F77DB
:104270008A87808D918D07C09924D5018C918F7785
:104280008A878D919C91880F892F881F990B919512
:104290008F778B87F501848980FF02C0F0E19F2A28
:1042A0000E94031E7B018C01862F8F778C8767E02D
:1042B00016950795F794E7946A95D1F78E2D8F7729
:1042C0008D8757E016950795F794E7945A95D1F79F
:1042D0008E2D8F778E8747E016950795F794E79494
:1042E0004A95D1F78E2D877089298F87AE01465F59
:1042F0005F4F6BE08FEF0E944620F9C00E94031EC3
:104300007B018C01DC01CB018F779070A070B070C5
:10431000F601248133274427552782179307A407E2
:10432000B50709F00EC1D801C70180789F73A0704E
:10433000B07037E0B695A795979587953A95D1F7E0
:10434000258133274427552782179307A407B507EC
:1043500009F0F7C0D801C7018070907CAF71B070D0
:104360002EE0B695A795979587952A95D1F7268142
:1043700033274427552782179307A407B50709F069
:10438000E0C080E090E0A0EEB0E0E822F9220A234D
:104390001B2375E116950795F794E7947A95D1F765
:1043A0002781822F9927AA27BB2787709070A0703A
:1043B000B070E816F9060A071B0709F0C2C0922E72
:1043C0009694969496948281A82FBB2783819927EF
:1043D0009695982F882797958795A82BB92B109796
:1043E00009F4AFC0092D112700FF09C0C5014A9685
:1043F000AC0160E070E0CD010E94C023DC011097A9
:1044000029F0BD01809134010E94761ED5018D9165
:104410009C91892B09F495C001FF93C0F501848913
:104420008160848B8EC0F6018281282F332783819F
:1044300099279695982F882797958795282B392B1C
:1044400030934B0320934A0352C0F6018281282FF8
:104450003327838199279695982F88279795879555
:10446000282B392B30934E0320934D038481809366
:104470005B03858180934F038681809350038091F5
:104480004C0381601CC0F6013296A1E5B3E094E0D4
:1044900081918D93915097FFFBCF80914C03826067
:1044A0000EC0D6011296E1E5F3E093E08D9185838D
:1044B0009150319697FFFACF80914C03846080939E
:1044C0004C0315C081E08093C70111C00E94E21E19
:1044D000F60182810E94390F0AC0F6018281882389
:1044E00021F00E94FB1DFC0184810E94D50CD601A5
:1044F0008C9199278F779070209134013327821700
:10450000930749F480914903882329F08091490356
:10451000815080934903F501848999279695879561
:104520009C012170307080FD04C0A90160E0C901C8
:1045300006C0F501468157816689808191810E947C
:10454000101FCE0101960E948D07892B09F0C8CD5E
:104550002F960FB6F894DEBF0FBECDBFDF91CF917F
:104560001F910F91FF90EF90DF90CF90BF90AF9091
:104570009F900895CF93DF93CDB7DEB726970FB600
:10458000F894DEBF0FBECDBF36E0FE01319611922A
:104590003A95E9F74983AE014F5F5F4F0E9446208D
:1045A00026960FB6F894DEBF0FBECDBFDF91CF9138
:1045B0000895CF93DF93CDB7DEB726970FB6F89463
:1045C000DEBF0FBECDBF26E0FE01319611922A95C7
:1045D000E9F7282F2F772983880F892F881F990BB8
:1045E00091958F778A83AE014F5F5F4F63E18FEFC5
:1045F0000E94462026960FB6F894DEBF0FBECDBFB0
:10460000DF91CF9108959F92AF92BF92CF92DF92A8
:10461000EF92FF920F931F93CF93DF93CDB7DEB747
:1046200026970FB6F894DEBF0FBECDBFFC018B01FD
:10463000942E6901672B11F0232B19F480E090E090
:1046400085C086E05E010894A11CB11CD5011D92B5
:104650008A95E9F754E1E52E8E2F8F778983EE0F47
:10466000EF2FEE1FFF0BF1958E2F8F778A8320E0BF
:104670008E2D99278631910501F18731910534F40A
:104680008431910549F04597C9F024C087319105DF
:1046900099F0489781F01EC0802F8F778B83C801D7
:1046A000880F892F881F990B91958F778C83892D7F
:1046B0008F778D830FC023E02D5F2D5F92E0D501B2
:1046C0001296F601E20FF11D80818D9391502F5FBC
:1046D00097FFF7CF10924B0310924A03FF2480916B
:1046E0004A0390914B03892B09F5AE014F5F5F4F51
:1046F0006E2D8FEF0E94462085E08093490306C00F
:1047000080914903882341F00E94320580914A0339
:1047100090914B03892BA1F3F39480914A039091DC
:104720004B03892B19F489E08F15F8F680914A0321
:1047300090914B03009751F0E0914A03F0914B03A5
:10474000E39488E18E1508F087CFCF0126960FB647
:10475000F894DEBF0FBECDBFDF91CF911F910F91B7
:10476000FF90EF90DF90CF90BF90AF909F90089513
:104770009A01462FBC0180E090E00E940323089537
:10478000DF92EF92FF920F931F93CF93DF93CDB7FA
:10479000DEB726970FB6F894DEBF0FBECDBF9C01E3
:1047A0007B018A0101978F5F934008F050C086E03B
:1047B000FE01319611928A95E9F7822F8F778983CE
:1047C000220F232F221F330B3195822F8F778A835D
:1047D00010924C03DD2480914C03873031F1AE01FF
:1047E0004F5F5F4F60E18FEF0E9446208FE0809324
:1047F000490306C080914903882331F00E943205A5
:1048000080914C038730B1F780914C03873029F0B9
:1048100082B7992788960E94FE09D39480914C0311
:10482000873019F089E08D15D0F680914C038730E0
:1048300021F480914F038F3769F4E114F10411F0F2
:10484000F70110820115110511F0F801108280E0C6
:1048500090E018C0E114F10421F080915B03F701AE
:1048600080830115110551F08BE0F801AFE4B3E04E
:104870000D9001928A95E1F7F801138680914D031E
:1048800090914E0326960FB6F894DEBF0FBECDBFB3
:10489000DF91CF911F910F91FF90EF90DF900895DE
:1048A0000F931F93CF93DF93CDB7DEB726970FB645
:1048B000F894DEBF0FBECDBF062F26E0FE01319675
:1048C00011922A95E9F7282F2F772983880F892FAE
:1048D000881F990B91958F778A838FEF9FEF909325
:1048E0004B0380934A0310E080914A0390914B035D
:1048F00097FF20C0AE014F5F5F4F602F8FEF0E9488
:10490000462085E08093490306C0809149038823AF
:1049100041F00E94320580914A0390914B03992304
:10492000A4F31F5F80914A0390914B0397FF02C04D
:104930001A3000F380914A0390914B0326960FB6EC
:10494000F894DEBF0FBECDBFDF91CF911F910F91C5
:10495000089561E10E945024089562E10E9450246C
:104960000895E199FECF9FBB8EBBE09A99278DB346
:1049700008954115510569F0DC01E199FECF7FBB37
:104980006EBBE09A6F5F7F4F0DB20D924150504069
:10499000B1F70895E199FECF9FBB8EBB6DBB0FB6FB
:1049A000F894E29AE19A0FBE0895DC0101C06D937C
:1049B00041505040E0F70895FB01DC0101900D9259
:1049C0000020E1F708950F931F93CF93DF93CDB7A6
:1049D000DEB72C970FB6F894DEBF0FBECDBF8C01AB
:1049E00036E03C8389839A832FEF3FE72D833E8314
:1049F000CE0101960E943525AF81B885A00FB11F69
:104A00001C922C960FB6F894DEBF0FBECDBFDF917F
:104A1000CF911F910F9108950F931F93CF93DF9321
:104A2000CDB7DEB72C970FB6F894DEBF0FBECDBF63
:104A30008C013EE03C8389839A832FEF3FE72D83EF
:104A40003E83CE0101960E943525AF81B885A00F27
:104A5000B11F1C922C960FB6F894DEBF0FBECDBFCF
:104A6000DF91CF911F910F9108952F923F924F9216
:104A70005F926F927F928F929F92AF92BF92CF92EE
:104A8000DF92EF92FF920F931F93CF93DF93CDB7F7
:104A9000DEB762970FB6F894DEBF0FBECDBFAA2473
:104AA000BB2465014C016D877E874F87588B44245A
:104AB0005524FC0146825782838181FD5BC28FEFC2
:104AC0009FEF6FC240FE44C2862D80538A30E0F4CF
:104AD000F0E36F1641F42A89222329F4772019F490
:104AE00080E091E08BC08AE09A89989F902D1124F4
:104AF000892F860D80538A8B882314F4EFE7EA8B85
:104B000043FC38C27A8836C243FE05C0FA89FF23C7
:104B100011F421E02A8B862D992787FD9095883600
:104B2000910554F5853691050CF06BC088359105DB
:104B300009F4D3C089359105B4F48B32910509F499
:104B400042C08C32910544F48032910509F43FC093
:104B5000839709F442C0F2C18D329105D9F18E9745
:104B600009F440C0EBC18336910509F454C0843682
:104B7000910509F478C0E2C18037910509F4A5C018
:104B80008137910584F48C369105B1F18D3691050C
:104B90002CF48936910509F466C0D0C18F36910591
:104BA00009F490C0CBC18537910509F498C08637C8
:104BB000910524F483379105B9F1C0C18837910577
:104BC00009F48BC0BBC180E190E0482A592AE0E299
:104BD000F0E005C080E890E011C0E0E4F0E04E2A8B
:104BE0005F2AC8C188E090E0482A592AEFEFFEEF1B
:104BF0004E225F221A8ABEC184E090E0482A592AD8
:104C0000B9C10F2EFFE3AF2EF02D7A940F2EF3E6ED
:104C10006F2EF02D3AC1EF85F889CF0102968F876C
:104C2000988BA0807A9431C1EF85F889CF010296E4
:104C30008F87988BA080B18043FE0BC0EA898E2FAE
:104C4000992787FD9095BC01C5010E941D28898B7D
:104C500007C0F50101900020E9F73197EA19E98BC7
:104C6000F9897F1A12C142FE0BC0EF85F889CF0186
:104C700004968F87988B20813181428153810DC0AA
:104C8000EF85F889CF0102968F87988B808191817B
:104C90009C01442737FD4095542F59016A01552343
:104CA00064F4E2E0F0E04E2A5F2AD094C094B0941D
:104CB000A094A11CB11CC11CD11C8FEB9FEF4822FA
:104CC00059222BC098E0998B0AC0E0E4F0E04E2A0C
:104CD0005F2A0F2EF8E76F2EF02DF0E1F98B42FEE0
:104CE0000BC0EF85F889CF0104968F87988B2081C0
:104CF0003181428153810BC0EF85F889CF01029643
:104D00008F87988B808191819C0144275527590179
:104D10006A01EFECFFEF4E225F221E010894211C76
:104D2000311CF989EF2EFF2400271127C601B50198
:104D3000A80197010E943428DC01CB01F101808396
:104D40008A301CF0860D815203C0F1018081805DA4
:104D5000F10181931F01C601B501A80197010E94CD
:104D6000342859016A012115310541055105F1F633
:104D7000CE010196A22CA81AC20182739070892BD1
:104D800009F07A9446FE0FC0872D992787FD9095EC
:104D9000F989F03131F40F2EFEEF7F2EF02D780ED1
:104DA00002C0782E7A9443FE12C08A89282F3327B6
:104DB00027FD30958A2D9927821793072CF0E7EF6E
:104DC000FFEF4E225F2203C0FA89FA19FA8B43FEE5
:104DD00003C02A89721A01C07A18C20180789170C2
:104DE000892B69F4872D7A9418164CF4B40180E26B
:104DF00090E00E94EA27872D7A941816BCF341FEB2
:104E000004C0B4018DE290E00BC044FE04C0B401C4
:104E10008BE290E005C045FE05C0B40180E290E061
:104E20000E94EA2746FE0FC0B40180E390E00E9492
:104E3000EA278989803139F4862D992787FD909555
:104E4000B4010E94EA2750FE0DC0872D7A941816EF
:104E50004CF4B40180E390E00E94EA27872D7A9415
:104E60001816BCF343FE11C08A89982F91509A8B73
:104E700018165CF4B40180E390E00E94EA278A8966
:104E8000E82FE150EA8B1816ACF3842D807869F492
:104E9000872D7A9418164CF4B40180E290E00E94B9
:104EA000EA27872D7A941816BCF3F3E66F1641F4BF
:104EB0008A2D992787FD9095B4010E94EA272DC07D
:104EC00023E76216B1F489898150898B8F3F29F1DC
:104ED000F5018081992787FD90950894A11CB11C4C
:104EE000B4010E94EA2799899150998B9F3F81F7DD
:104EF00014C0CE0101962816390679F08E010F5F95
:104F00001F4FF10182911F01992787FD9095B401F0
:104F10000E94EA2720163106A1F7842D8078A9F097
:104F2000872D7A9418168CF4B40180E290E00E94E8
:104F3000EA27872D7A941816BCF307C0862D992787
:104F400087FD9095B4010E94EA274424552412C09D
:104F5000F5E26F1641F44424552443941A8A7A8862
:104F60002AE0298B07C0862D992787FD9095B401EB
:104F70000E94EA27F401838183FF08C0ED85FE8546
:104F8000CF0101968D879E87649005C0ED85FE85D3
:104F90006190ED87FE87662009F094CDF40186814B
:104FA000978162960FB6F894DEBF0FBECDBFDF913A
:104FB000CF911F910F91FF90EF90DF90CF90BF9016
:104FC000AF909F908F907F906F905F904F903F90A9
:104FD0002F9008950F931F93CF93DF938C01EB01D4
:104FE0008B81992781FF22C082FF14C02E813F81CF
:104FF0004C815D81241735073CF4A881B9810D935C
:10500000A883B9832E813F812F5F3F4F2E833F833B
:10501000C8010EC0E885F985802F0995892B31F4E8
:10502000EE81FF813196EE83FF83F2CF8FEF9FEF0A
:10503000DF91CF911F910F910895FC016150704055
:1050400001900110D8F7809590958E0F9F1F0895BD
:10505000991B79E004C0991F961708F0961B881FCA
:105060007A95C9F780950895A1E21A2EAA1BBB1B59
:10507000FD010DC0AA1FBB1FEE1FFF1FA217B30724
:10508000E407F50720F0A21BB30BE40BF50B661F3A
:10509000771F881F991F1A9469F7609570958095FE
:0C50A00090959B01AC01BD01CF0108956B
:1050AC00FFFF00010000FF00004619FF0000E4189C
:1050BC00FF0000FD14FF00004315FF01004F17FF18
:1050CC0001005515FF01007816FF01004C18FF0177
:0650DC00009D18FFFF001B
:00000001FF
